:100000000C945B000C9483000C9483000C9483008C
:100010000C9483000C9483000C9483000C94830054
:100020000C9483000C9483000C9483000C94830044
:100030000C9483000C9483000C9483000C94830034
:100040000C941A030C9483000C949B050C9483006D
:100050000C9483000C9483000C9483000C94830014
:100060000C9483000C948300000024272A000025B0
:10007000282B000023262904040404040404040299
:100080000202020202030303030303010204081035
:100090002040800102040810200102040810200002
:1000A0000000070002010000030406000000000039
:1000B00000000000720111241FBECFEFD4E0DEBFAC
:1000C000CDBF11E0A0E0B1E0E8E8FCE002C005909F
:1000D0000D92AA30B107D9F711E0AAE0B1E001C052
:1000E0001D92A03CB107E1F710E0C6EBD0E004C0E0
:1000F0002297FE010E943E06C43BD107C9F70E9429
:100100006B010C9442060C940000CF93DF93109285
:10011000310110923001C1E0D0E04EC06AE070E0E1
:1001200080E090E00E948503809130010E94FA03F4
:10013000803891057CF0E0913001F0913101EE0FB3
:10014000FF1FE65FFE4F80819181019761F511826B
:10015000108229C0809130010E94FA0380389105F5
:1001600014F52091300130913101220F331FF90134
:10017000E65FFE4F80819181892BA9F4A901662752
:1001800057FD6095762F20E030E082E391E00E94F9
:10019000FA02E0913001F0913101EE0FFF1FE65FAE
:1001A000FE4FD183C083809130019091310101963F
:1001B0009093310180933001809130019091310111
:1001C00006970CF4ABCF82E090E0909331018093DE
:1001D0003001C1E0D0E04EC06AE070E080E090E025
:1001E0000E948503809130010E94D504019779F423
:1001F000E0913001F0913101EE0FFF1FEA5EFE4FFA
:1002000080819181019769F5118210822AC08091C5
:1002100030010E94D504892B21F5209130013091C5
:100220003101220F331FF901EA5EFE4F8081918177
:10023000892BB9F4285F3F4FA901662757FD6095C8
:10024000762F20E030E082E391E00E94FA02E09114
:100250003001F0913101EE0FFF1FEA5EFE4FD183B6
:10026000C0838091300190913101019690933101CA
:100270008093300180913001909131010C970CF402
:10028000ABCFDF91CF91089540E052EC61E070E098
:1002900082E391E00E94860164E670E080E090E0F5
:1002A0000E94850310923101109230010CC060E071
:1002B0000E946C04809130019091310101969093DD
:1002C00031018093300180913001909131018C3067
:1002D00091056CF308950E94BD030E9444010E94A1
:1002E0008500FDCF86E091E0909333018093320149
:1002F0000895862F0E945A0508950E949205089538
:100300000E94730508950E9462050895CB01BA0109
:100310000E9421050895DC01ED91FC910190F0818E
:10032000E02D09950895DC01ED91FC910190F0819B
:10033000E02D099508950F931F93CF93DF938C01C0
:10034000EB0109C02196D801ED91FC910190F0815B
:10035000E02DC801099568816623A1F7DF91CF914F
:100360001F910F9108950F931F938C01DC01ED9164
:10037000FC910190F081E02D6DE00995D801ED919F
:10038000FC910190F081E02D6AE0C80109951F9170
:100390000F9108950F931F938C01DC01ED91FC9157
:1003A0000190F081E02D0995C8010E94B3011F91D1
:1003B0000F9108950F931F938C010E949B01C80118
:1003C0000E94B3011F910F9108950F931F938C0109
:1003D000DC01ED91FC910190F081E02D0995C801BF
:1003E0000E94B3011F910F9108952F923F924F9257
:1003F0005F926F927F928F929F92AF92BF92CF92B5
:10040000DF92EF92FF920F931F93DF93CF93CDB7BD
:10041000DEB7A0970FB6F894DEBF0FBECDBF1C01AC
:100420006A017B01411551056105710549F4DC0143
:10043000ED91FC910190F081E02D60E3099554C0AD
:10044000882499245401422E55246624772401E0FF
:1004500010E00C0F1D1F080D191DC701B601A301E7
:1004600092010E94EB05F80160830894811C911CA5
:10047000A11CB11CC701B601A30192010E94EB05AA
:10048000C901DA016C017D01C114D104E104F10458
:10049000F1F681E0E82EF12CEC0EFD1EE80CF91CC3
:1004A0003E010894611C711CD501C4010197A1098A
:1004B000B1096C01C818D90814C0F601EE0DFF1D72
:1004C00060816A3010F4605D01C0695CD101ED911A
:1004D000FC910190F081E02DC10109950894E1089B
:1004E000F1086E147F0449F7A0960FB6F894DEBFAA
:1004F0000FBECDBFCF91DF911F910F91FF90EF9075
:10050000DF90CF90BF90AF909F908F907F906F9033
:100510005F904F903F902F9008952AE00E94F50140
:1005200008950F931F938C010E948D02C8010E94B1
:10053000B3011F910F910895AB0160E070E00E943C
:100540008D0208950F931F938C01AB0160E070E062
:100550000E948D02C8010E94B3011F910F9108955E
:10056000EF92FF920F931F93CF93DF93EC017A01E9
:100570008B0177FF0FC0E881F9810190F081E02DB8
:100580006DE2099510950095F094E094E11CF11C42
:10059000011D111D2AE0B801A701CE010E94F5013D
:1005A000DF91CF911F910F91FF90EF9008950F93DE
:1005B0001F938C010E94B002C8010E94B3011F91D9
:1005C0000F910895AB01662757FD6095762F0E9425
:1005D000B00208950F931F938C01AB01662757FD5E
:1005E0006095762F0E94B002C8010E94B3011F914E
:1005F0000F910895DC012115310541F4ED91FC9135
:100600000190F081E02D642F099508952A3031057D
:1006100019F40E94B00208950E94F50108950F9305
:100620001F938C010E94FA02C8010E94B3011F911E
:100630000F9108951F920F920FB60F9211242F93CE
:100640008F939F93AF93BF93809134019091350125
:10065000A0913601B09137018050904CAF4FBF4F01
:100660008093340190933501A0933601B093370104
:1006700027C08091340190913501A0913601B0914D
:10068000370180589E43A040B0408093340190933E
:100690003501A0933601B0933701809138019091D4
:1006A0003901A0913A01B0913B010196A11DB11D04
:1006B0008093380190933901A0933A01B0933B01A4
:1006C0008091340190913501A0913601B0913701AC
:1006D00081589E43A040B04060F6BF91AF919F917A
:1006E0008F912F910F900FBE0F901F9018958FB77D
:1006F000F894209138013091390140913A0150919C
:100700003B018FBFB901CA010895EF92FF920F9389
:100710001F937B018C018FB7F89440913801509161
:10072000390160913A0170913B018FBF2FB7F89466
:100730008091380190913901A0913A01B0913B012B
:100740002FBF841B950BA60BB70B8E159F05A0071B
:10075000B10760F31F910F91FF90EF9008950197FB
:1007600059F0FC01EE0FFF1FEE0FFF1F32978FB7FE
:10077000F8943197F1F78FBF0895789484B582602B
:1007800084BD84B5816084BD85B5826085BD85B535
:10079000816085BDEEE6F0E0808181608083E1E8E4
:1007A000F0E0808182608083808181608083E0E8E6
:1007B000F0E0808181608083E1EBF0E08081846003
:1007C0008083E0EBF0E0808181608083EAE7F0E005
:1007D0008081846080838081826080838081816069
:1007E00080838081806880831092C1000895809307
:1007F000080108958F70909108019295990F990FB3
:10080000907C982B90937C0080917A0080648093F8
:100810007A0080917A0086FDFCCF2091780040918B
:100820007900942F80E030E0282B392BC9010895FE
:100830001F93CF93DF93182FEB0161E00E946C04AC
:10084000E12FF0E0E156FF4F8491833051F4809125
:100850008000806880938000D0938900C0938800D6
:1008600037C0843051F48091800080628093800092
:10087000D0938B00C0938A002BC0813029F484B5BB
:10088000806884BDC7BD24C0823029F484B58062ED
:1008900084BDC8BD1DC0863041F48091B000806821
:1008A0008093B000C093B30013C0873041F48091AF
:1008B000B00080628093B000C093B40009C0C0381B
:1008C000D10514F460E001C061E0812F0E948A0428
:1008D000DF91CF911F910895282F30E0C9018557EE
:1008E0009F4FFC01949129583F4FF901849188232F
:1008F00081F0E82FF0E0E859FF4FE491F0E0662343
:1009000029F4808190958923808308958081892BA3
:1009100080830895482F50E0CA0181569F4FFC0103
:100920002491CA0185579F4FFC01949149585F4F0C
:10093000FA0134913323C1F1222331F1233021F420
:10094000809180008F7705C0243031F48091800041
:100950008F7D8093800018C0213019F484B58F7783
:1009600004C0223021F484B58F7D84BD0DC02630B3
:1009700021F48091B0008F7705C0273029F4809151
:10098000B0008F7D8093B000E32FF0E0E359FF4F7C
:10099000E491F0E0662329F4808190958923808397
:1009A00008958081892B80830895482F50E0CA01E3
:1009B00081569F4FFC012491CA0185579F4FFC012E
:1009C000949149585F4FFA013491332319F420E090
:1009D00030E035C0222331F1233021F480918000B2
:1009E0008F7705C0243031F4809180008F7D809313
:1009F000800018C0213019F484B58F7704C02230EC
:100A000021F484B58F7D84BD0DC0263021F4809102
:100A1000B0008F7705C0273029F48091B0008F7D1A
:100A20008093B000E32FF0E0EE58FF4FE491F0E048
:100A3000808120E030E0892311F021E030E0C9011D
:100A40000895EF92FF920F931F937B018C0122E098
:100A500030E040E050E00E940D06205C3D4B404FEE
:100A60005F4FCA01B901A80197010E940D06C90193
:100A7000DA010197A109B109292F3A2F4B2F5527E8
:100A800047FD5A950196A11DB11D2093C5008150C7
:100A90008093C400E1ECF0E08081806180838081FC
:100AA000886080838081806880831F910F91FF9090
:100AB000EF900895982F8091C00085FFFCCF909310
:100AC000C600089580913C0190913D0180589F4F50
:100AD00020913E0130913F01821B930B60E870E052
:100AE0000E94D805089540913E0150913F018091A8
:100AF0003C0190913D018417950719F42FEF3FEFCA
:100B00000FC0FA01E05CFE4F2081CA01019660E847
:100B100070E00E94D80590933F0180933E0130E041
:100B2000C901089580913E0190913F0190933D014C
:100B300080933C0108951F920F920FB60F921124DB
:100B40002F933F934F935F936F937F938F939F93D5
:100B5000AF93BF93EF93FF934091C600E0913C01A8
:100B6000F0913D01CF01019660E870E00E94D80548
:100B70009C0180913E0190913F012817390739F07F
:100B8000E05CFE4F408330933D0120933C01FF9198
:100B9000EF91BF91AF919F918F917F916F915F91F5
:100BA0004F913F912F910F900FBE0F901F9018956E
:100BB00097FB092E07260AD077FD04D049D006D02E
:100BC00000201AF4709561957F4F0895F6F790957F
:100BD00081959F4F0895A1E21A2EAA1BBB1BFD0110
:100BE0000DC0AA1FBB1FEE1FFF1FA217B307E4070C
:100BF000F50720F0A21BB30BE40BF50B661F771F64
:100C0000881F991F1A9469F7609570958095909543
:100C10009B01AC01BD01CF01089597FB092E05266C
:100C20000ED057FD04D0D7DF0AD0001C38F4509501
:100C30004095309521953F4F4F4F5F4F0895F6F700
:100C400090958095709561957F4F8F4F9F4F089538
:100C5000AA1BBB1B51E107C0AA1FBB1FA617B707E2
:100C600010F0A61BB70B881F991F5A95A9F78095FE
:100C70009095BC01CD010895EE0FFF1F0590F491F2
:080C8000E02D0994F894FFCF68
:0A0C88000A000000000079010100DD
:00000001FF
